:1000000000308A0019280000223084008313000881
:10001000031918280130F800F701F70B0D28F80B29
:100020000C284A30F700F70B13281628800B0A28F3
:100030000800840183131F308305613083168F000D
:100040000F0803170908C039890003131F129F12F4
:100050000030031788008312870188018901FF306F
:100060000313A000831603170908C039890003137E
:100070001F129F12003003178800831203131F13EF
:100080009F1383169F1383121F149412A01220082B
:100090008316870083122016200883168700831298
:1000A000A0112008831687000130831294000030CD
:1000B000831694000108C739083881008312900123
:1000C0000030F80092000030831692008312201551
:1000D0002008831687008312970183169B019C01D9
:1000E00001309D008312031787018801890183165F
:1000F00003130813831208130430A100FA30A2007E
:100100000420A10B7E2883160813831208170430DD
:10011000A100FA30A2000420A10B89280317772838
:0201200063007A
:04400E00F52CFF3F4F
:00000001FF
